:1000000012C02CC02BC0EAC65DC628C027C026C0BF
:1000100025C024C023C022C021C020C01FC01EC0D4
:100020001DC01CC01BC011241FBECFE5D4E0DEBF25
:10003000CDBF10E0A0E6B0E0E2E3FAE102C0059037
:100040000D92AC3BB107D9F710E0ACEBB0E001C0CA
:100050001D92A13FB107E1F79EDAE9CCD1CF61153E
:100060007105E1F0E82FF92F20E030E080E0B8E002
:10007000A8E141919B2F542F582750FF04C08A2795
:100080008695806801C08695915011F04695F3CF12
:100090002F5F3F4F6217730761F7089580E008955F
:1000A000DC01CB0181159105A105B10529F0815035
:1000B0009040A040B040D9F70895282F30E0207735
:1000C0003070A901440F551F220F331F220F331F19
:1000D000220F331F240F351F35952795359527950A
:1000E00035952795359527958F70820F089520E0D7
:1000F00030E0A0E0BAE06B2F52DC492F50E0F9016C
:10010000EE0FFF1FEE0FFF1F02C0440F551FEA95B1
:10011000E2F7A42B2F5F3F4F2430310561F78A2F80
:100120000895DAD280EDECD28EE0EAD280E0E8D217
:10013000DFD20895EF92FF920F931F93CF93DF9337
:100140007C018B01EA01C8D280EDDAD280E0D8D2FE
:10015000CFD2C2D281EDD4D281E0F0D2AEDF88839B
:10016000C7D2BAD281EDCCD281E0E8D2A6DFF801C5
:100170008083BED2B1D281EDC3D281E0DFD29DDFD8
:10018000F7018083B5D2DF91CF911F910F91FF903E
:10019000EF900895FF920F931F93182F062FF42EC0
:1001A0009BD280EDADD280E0ABD28F2DA0DFA8D264
:1001B000802F9DDFA5D2812F9ADFA2D299D21F91E5
:1001C0000F91FF900895EF92FF920F931F93CF939B
:1001D000DF938C017B01EA017FD280ED91D284E034
:1001E0008FD286D279D281ED8BD281E0A7D265DF22
:1001F000F80180837DD270D281ED82D281E09ED2DF
:100200005CDFF701808374D267D281ED79D281E01F
:1002100095D253DF88836CD2DF91CF911F910F91DC
:10022000FF90EF900895FF920F931F93F82E062FE3
:10023000142F52D280ED64D284E062D28F2D57DF2A
:100240005FD2802F54DF5CD2812F51DF59D250D240
:100250001F910F91FF9008951F93182F3DD280EDAD
:100260004FD2812F4DD238D281ED4AD280E066D272
:10027000182F3ED2812F1F9108950F931F93082F9F
:10028000162F2AD280ED3CD2802F3AD2812F38D23D
:100290002FD21F910F9108950F931F93CF93DF9348
:1002A000FB01E801608170E0B181A0E06A2B7B2B4B
:1002B000803179F46E7FDB01AA0FBB1FAA0FBB1F31
:1002C000AA0FBB1F96816CE070E0691B71096A0F71
:1002D0007B1F77233CF491E0DA019C937095619544
:1002E0007F4F02C0DA011C92883289F4848190E049
:1002F000AC01407650704036510549F086FF02C08F
:100300006E7F05C085FF02C06C7F01C0687FCB0196
:10031000929582958F7089279F708927F901808334
:100320006F70688380E0DF91CF911F910F910895E6
:100330000F931F93DF93CF93CDB7DEB728970FB6F8
:10034000F894DEBF0FBECDBF182F062FDE01119629
:10035000E0E6F0E088E001900D928150E1F7642F33
:1003600070E021E732E0629FC001639F900D729FB1
:10037000900D112468EE73E032DB9B016AE0069F6A
:10038000B0011124620F731F112381F48981841736
:1003900039F0FE013296CE0109962191241719F405
:1003A0006F5F7F4F03C0E817F907B9F7862F972FC4
:1003B00028960FB6F894DEBF0FBECDBFCF91DF9168
:1003C0001F910F910895882319F0709561957F4FC3
:1003D000442319F0309521953F4F6217730734F08D
:1003E00081E0261737071CF080E008958FEF08950D
:1003F0000F931F93CF93DF93EC018B018881B8019A
:1004000064DA888381508D3F30F4F801808188322E
:1004100011F0803199F7DF91CF911F910F910895DD
:100420001F93CF93DF93EC01A2D984EBBE019DDA39
:1004300081E0F8D9182F9BD981E0112309F480E0DD
:10044000DF91CF911F9108951F93CF93DF93182FC2
:10045000EB018DD95BD9882341F084E4BE0185DAB4
:10046000113029F05CD980E003C082E001C080E057
:10047000DF91CF911F9108956F927F928F929F92FB
:10048000AF92BF92CF92DF92EF92FF920F931F93A2
:10049000DF93CF93CDB7DEB729970FB6F894DEBFC1
:1004A0000FBECDBF6C014B013A01590160D98EEBF3
:1004B000B6015BDA8E010F5F1F4F0F2EFAE0EF2EB1
:1004C000FF24F02DEC0EFD1EFDD9F80181938F0164
:1004D000EE15FF05C9F7CE01019669E070E0BFDDBA
:1004E000882359F4F6018081BE016F5F7F4FA4011C
:1004F00093018501D1DE80E001C083E029960FB62B
:10050000F894DEBF0FBECDBFCF91DF911F910F9149
:10051000FF90EF90DF90CF90BF90AF909F908F9023
:100520007F906F9008957F928F929F92AF92BF922B
:10053000CF92DF92EF92FF920F931F93DF93CF93AF
:10054000CDB7DEB729970FB6F894DEBF0FBECDBF8B
:10055000782E5B014A0169018EEB60E070E005DAFC
:100560008E010F5F1F4F0F2EFAE0EF2EFF24F02DAC
:10057000EC0EFD1EA7D9F80181938F01EE15FF0542
:10058000C9F7CE01019669E070E069DD882351F476
:10059000872DBE016F5F7F4FA501940186017CDE30
:1005A00080E001C083E029960FB6F894DEBF0FBE4D
:1005B000CDBFCF91DF911F910F91FF90EF90DF9012
:1005C000CF90BF90AF909F908F907F900895FF92B3
:1005D0000F931F93CF93DF93EC01062F142FF22E6E
:1005E000C6D894D8882371F08EE4BE01BED9802F7E
:1005F00059D9812F57D98881883231F48F2D52D91A
:1006000080E003C081E001C080E0DF91CF911F91C5
:100610000F91FF900895EF92FF920F931F93CF9346
:10062000DF93EC01062F172FA2D870D8882379F01A
:100630008EEBBE019AD9E02EE7017E01F12EE70193
:1006400019E040D989931150E1F780E001C081E0C1
:10065000DF91CF911F910F91FF90EF9008951F931D
:10066000CF93DF93182FEB0182D850D88823A9F0BD
:1006700088E4BE017AD9113049F051D860E27EE4B5
:1006800080E090E00DDD5ED880E008C060E27EE4AE
:1006900080E090E005DD80E001C082E0DF91CF9155
:1006A0001F910895CF93DF93EC0161D82FD8882351
:1006B00051F088EBBE0159D960E27EE480E090E021
:1006C000EFDC80E001C081E0DF91CF910895969842
:1006D00097988E988F9808958E9A000008958F9A13
:1006E00000008E9800008F9800008E9A00000895F8
:1006F0008F9A8E9A00008F9800008E9800000895BF
:1007000098E08F9A882314F48E9801C08E9A000086
:100710008F980000915011F0880FF3CF8F9A8E9828
:1007200000008F98000080B382958695869583702F
:1007300080FF02C08FEF089580E00895382F8F9AD0
:100740008E9800008F98000090B39295969596959C
:100750009370892F817097E08F9A00008F98000026
:10076000880F20B326FD81609150B1F78F9A332313
:1007700011F48E9A01C08E9800008F9800000895A1
:100780001F93413059F4182F110F160F02C0B0DF1C
:10079000A3DF812FB5DF8F3FD1F303C0880F860F12
:1007A000AFDF1F910895AF92BF92DF92EF92FF9259
:1007B0000F931F93DF93CF93CDB7DEB729970FB673
:1007C000F894DEBF0FBECDBF8FEF8987EE24FF24E4
:1007D0008E01075F1F4F5E010894A11CB11CDE2C27
:1007E000C801B50105DE89858F3F31F48093B900DA
:1007F00081E08093BA0023C08E3F39F48FEF80935D
:10080000B90081E08093BA001AC0F501D701AA0FA0
:10081000BB1FAA0FBB1FAA0FBB1FA752BF4F8191BF
:100820008D93E017F107D9F7D3948985882339F0A0
:100830000894E11CF11C82E0E816F10481F68D2D8C
:1008400029960FB6F894DEBF0FBECDBFCF91DF91D2
:100850001F910F91FF90EF90DF90BF90AF900895A0
:100860001F93262F9091C000992399F53AE0632FAA
:1008700096D88093C5009093C600822F90D880931D
:10088000C7009093C800842F8AD88093C9009093A2
:10089000CA00E5ECF0E080E090E04AE750E021EDAE
:1008A00030E011E07191DA01A80FB91F6C91761751
:1008B00029F0D901A80FB91F1C9304C0D901A80FB2
:1008C000B91F1C9201968630910561F71092C10004
:1008D0000CC01092D1001092D2001092D30010924E
:1008E000D4001092D5001092D6001F9108959F92C7
:1008F000AF92BF92CF92DF92EF92FF920F931F932E
:10090000CF93DF93262F3AE0632F49D88093C50019
:100910009093C600822F43D88093C7009093C8005D
:10092000842F3DD88093C9009093CA0025EC30E015
:10093000AA24BB244AE750E061ED70E0EE246894FD
:10094000E1F80F2EF3E0FF2EF02D0F2EF9E09F2E91
:10095000F02DF501E9011881DA01AA0DBB1DAC915A
:10096000A11720F4DB01AA0DBB1DEC92DA01AE0F3A
:10097000BF1FAC911A1720F4DB01AE0FBF1FFC9212
:10098000192DDB01AE0FBF1FE40FF51FDC900D2DFD
:10099000023039F4C080D880CD1419F0D080D394BF
:1009A000D082DC908D2D833039F4C080D880CD1476
:1009B00019F0D080DA94D082C080D880CD1441F074
:1009C0008BE594E40197F1F700C000001150F1F6B7
:1009D0000894A11CB11C2F5F3F4F96E0A916B104EB
:1009E00009F0B7CFDF91CF911F910F91FF90EF905A
:1009F000DF90CF90BF90AF909F900895AF92BF923D
:100A0000DF92EF92FF920F931F93CF93DF937C01BE
:100A100085E090E0ABE7B0E0FD013197AF014E5FBC
:100A20005F4F9F012D5F3F4FAA24BB246894A2F81B
:100A3000AE0EBF1E8F010B5F1F4F0F2EFAE0DF2E91
:100A4000F02D6C916083EA0168816C93E901688103
:100A5000EA016883E5016881E9016883E80168814A
:100A6000E5016883BF01680F791FEB01D882C7EAEF
:100A7000D1E62197F1F700C00000019711F78AE055
:100A800080937A00C70164E670E095D7E62F2AE0EC
:100A900030E0C701B9018FD7482FCB01B9018BD7FF
:100AA000642F25E030E04AE750E09AE0DA01A20F37
:100AB000B31FEC93D9011196A40FB51F8C93D901E4
:100AC0001296A40FB51F6C93D9011396A40FB51FEE
:100AD0009C93A7EAB1E61197F1F700C000002150FE
:100AE00030402130310511F78091BA00813031F466
:100AF000809186008093730010927A00DF91CF91ED
:100B00001F910F91FF90EF90DF90BF90AF900895ED
:100B1000CF92DF92FF920F931F93CF93DF93809139
:100B20007A008823D9F580E090E0EEE7F0E08F01CD
:100B30000F5F1F4FAF01415050409F012250304086
:100B4000EF0123970F2EFCEFCF2EFFEFDF2EF02DBE
:100B5000CE0EDF1E0F2EFAE0FF2EF02D6081D801A1
:100B60006C93DA016C916083D9016C91DA016C931A
:100B70006881D9016C93D6016C916883B601680FC6
:100B8000791FDB01FC92A7EAB1E61197F1F700C0EB
:100B9000000001968630910509F736C080E090E0AC
:100BA000EEE7F0E0BF016F5F7F4FEF0121970F2E5F
:100BB000FEEFCF2EFFEFDF2EF02DCE0EDF1EAF01AA
:100BC000435050408F01045010400F2EFAE0FF2E8A
:100BD000F02D2081DB012C9328812083D6012C91DC
:100BE0002883DA012C91D6012C939801280F391F04
:100BF000D901FC92A7EAB1E61197F1F700C0000015
:100C000001968430910529F78FEC90E068ED70E053
:100C10004EEC50E08FDA8091CF0025EC30E04AE0D6
:100C2000642FBDD68093C5009093C6008091D800F4
:100C3000B6D68093C7009093C8008091CE00AFD6FF
:100C40008093C9009093CA00F9013696B901AEE7C6
:100C5000B0E08D010F5F1F4FAD01415050409D012D
:100C600022503040CD0103970F2EFCEFCF2EFFEF27
:100C7000DF2EF02DCA0EDB1EFC90E801F882EA019F
:100C8000F880FC92E901F880EA01F882EC01F88032
:100C9000E901F882E601F880EC01F882F290E601C1
:100CA000F882C7EAD1E62197F1F700C00000E61705
:100CB000F70711F7DF91CF911F910F91FF90DF9010
:100CC000CF9008951F920F920FB60F921124DF92CA
:100CD000EF92FF920F931F932F933F934F935F9346
:100CE0006F937F938F939F93AF93BF93CF93DF9334
:100CF000EF93FF9315BA949893988091C200E3E71D
:100D0000F0E0E80FF11D808183BD8091C100893141
:100D100008F04CC08091C3008F5F8093C300823184
:100D200009F044C01092C300F090C100E09085002B
:100D3000CF2DD0E080E090E041ED50E0DE01A05604
:100D4000BF4F63E770E0C957DF4F0AE710E09C012F
:100D5000FA01E80FF91FE081E13011F0FF2071F492
:100D6000EE2DE13031F4D880FB01E20FF31FD08289
:100D700005C0DC90FB01E20FF31FD082FF2DFC3099
:100D800061F4E091C000EE2341F4FC01EB53FF4F0E
:100D9000D080200F311FF901D08201968630910555
:100DA000B1F68091C1008F5F8093C100FF91EF91F8
:100DB000DF91CF91BF91AF919F918F917F916F9173
:100DC0005F914F913F912F911F910F91FF90EF9065
:100DD000DF900F900FBE0F901F9018951F920F92EB
:100DE0000FB60F9211248F939F93EF93FF938091EF
:100DF000C2008630B0F4EAE7F0E0E80FF11D808130
:100E0000E8E6F0E0E80FF11D808188BB81E090E02A
:100E10000090C20002C0880F991F0A94E2F785BBB8
:100E200008C0863031F480918400813011F4949AA6
:100E3000939A8091C2008F5F8093C200873010F038
:100E40001092C200FF91EF919F918F910F900FBE72
:100E50000F901F901895CF93DF93EC01809186003F
:100E60008093730080937400809375008093760064
:100E7000809377008093780081E060E070E0E4DAAE
:100E8000C752DF4F88818093CB006AEB70E049EB5B
:100E900050E02DEC30E047DB882331F08FEF80937A
:100EA000B90081E08093BA008091BA006091B900E6
:100EB0004091CD003DDAA2DDDF91CF9108958FEC16
:100EC00090E068ED70E04EEC50E034D98091CF00B6
:100ED0006091D8004091CE00C3DC089587ED90E08A
:100EE00069EE70E040ED50E06ED98091860080930D
:100EF00073008093740080937500809376008093D4
:100F00007700809378008091D7006091E90040914C
:100F1000D000EDDC089580918300813061F0813054
:100F200030F0823041F1833009F0AAC05CC0C7DFE5
:100F30001092BD0008958091BD00893708F4BFDF8D
:100F40008091BD00893709F4C9DF8091BD008338E5
:100F500008F496C08FEC90E068ED70E04EEC50E045
:100F6000E9D88091CF006091D8004091CE00BFDCDD
:100F70001092BD0008958091BD00893708F49FDF6D
:100F80008091CC00882319F41092BD0010C08130EC
:100F900071F48091BD00893719F480E090E05BDF47
:100FA0008091BD00833818F0B3DD1092BD008091B0
:100FB000CC00823009F064C08091BD00893719F4FB
:100FC00080E090E048DF8091BD00833819F481E033
:100FD00090E041DF8091BD008D3808F451C098DD6C
:100FE0001092BD0008958091BD00893708F467DF35
:100FF0008091BD00893709F471DF8091CC0088238E
:10100000A1F48091BD00833880F08FEC90E068ED12
:1010100070E04EEC50E08ED88091CF006091D80007
:101020004091CE0064DC1092BD008091CC008130F4
:1010300071F48091BD00833819F480E090E00BDFFB
:101040008091BD008D3818F063DD1092BD00809155
:10105000CC008230A9F48091BD00833819F480E07F
:1010600090E0F9DE8091BD008D3819F481E090E0C8
:10107000F2DE8091BD00873918F04ADD1092BD0084
:1010800008958091BE008823D9F08091C0008330FC
:10109000B8F48091CF002AE0622F81D480937A0047
:1010A00090937B008091D8007AD480937C009093B9
:1010B0007D008091CE0073D480937E0090937F005A
:1010C0008091BE008823D9F08091C0008330B8F0B1
:1010D0008091D7002AE0622F62D480937A009093A7
:1010E0007B008091E9005BD480937C0090937D002D
:1010F0008091D00054D480937E0090937F008091A3
:10110000C000833009F48FC0843030F4813059F04E
:10111000823009F03AC147C0843009F4C3C0853039
:1011200009F033C1FEC0819912C08091CF008F5F5A
:101130008093CF00883110F01092CF008FE996E8AD
:10114000A1E081509040A040E1F700C000008299EA
:1011500015C08091CF0081508093CF00829905C047
:10116000882319F487E18093CF008FE996E8A1E006
:1011700081509040A040E1F700C00000B09904C049
:10118000829B02C0819909C08091CF006AE007D498
:1011900080937A0090937B0008958AE080937A0090
:1011A00080937B000895819912C08091D8008F5F51
:1011B0008093D8008C3310F01092D8008FE996E815
:1011C000A1E081509040A040E1F700C0000082996A
:1011D00015C08091D80081508093D800829905C0B5
:1011E000882319F48BE38093D8008FE996E8A1E077
:1011F00081509040A040E1F700C00000B09904C0C9
:10120000829B02C0819909C08091D8006AE0C7D34F
:1012100080937C0090937D0008958AE080937C0009
:1012200080937D000895819913C08091D7008F5FCE
:101230008093D700803218F081E08093D7008FE947
:1012400096E8A1E081509040A040E1F700C0000086
:10125000829913C08091D70081508093D700882352
:1012600019F48FE18093D7008FE996E8A1E08150CF
:101270009040A040E1F700C00000B09904C0829BFC
:1012800002C0819909C08091D7006AE088D3809319
:101290007A0090937B0008958AE080937A0080938F
:1012A0007B000895819913C08091E9008F5F80933E
:1012B000E9008D3018F081E08093E9008FE996E82D
:1012C000A1E081509040A040E1F700C00000829969
:1012D00013C08091E90081508093E900882319F4BC
:1012E0008CE08093E9008FE996E8A1E0815090407E
:1012F000A040E1F700C00000B09904C0829B02C08A
:10130000819909C08091E9006AE049D380937C000B
:1013100090937D0008958AE080937C0080937D0007
:10132000089581990EC08091D0008F5F8093D00086
:101330008FE996E8A1E081509040A040E1F700C01D
:10134000000082990EC08091D00081508093D0001F
:101350008FE996E8A1E081509040A040E1F700C0FD
:101360000000B09904C0829B02C0819909C080919D
:10137000D0006AE014D380937E0090937F0008959C
:101380008AE080937E0080937F000895819926C033
:101390008091C000882329F48091BF008F5F8093E3
:1013A000BF008091BF008A3079F480918400813041
:1013B00019F41092840003C081E08093840060914E
:1013C000840080E090E026D32FE936E841E0215008
:1013D00030404040E1F700C000001BC08091BF00DA
:1013E0008823A9F08091BF008A3088F48AE0809336
:1013F000C00074DD8FE79AE1A6E081509040A040E4
:10140000E1F700C000001092C0001092BF001092DF
:10141000BF00829929C08091C000882329F58AE005
:101420008093C0008091CC00882319F080E090E088
:1014300012DD2FE73AE146E0215030404040E1F72D
:1014400000C000008091CC00823061F481E090E027
:1014500002DD8FE79AE1A6E081509040A040E1F7DD
:1014600000C000001092C00080995BC08091BE0057
:101470008F5F8093BE008091C000823031F48091F4
:10148000CF006091D80040E085D68091BE008130C9
:1014900049F48091C000882329F08091C0008F5FBB
:1014A0008093C0008091BE008A30A1F48091C0007A
:1014B000882381F481E08093C000109284002FE99A
:1014C00036E841E0215030404040E1F700C00000E4
:1014D000809384008091C0008630C8F01092840010
:1014E0008FE996E8A1E081509040A040E1F700C06C
:1014F000000081E0809384008091D7006091E90032
:101500004091D00090D61092C0001092BE002FE9FA
:1015100036E841E0215030404040E1F700C0000093
:1015200008958091C000882399F58091BE0088239A
:1015300079F1809183008F5F809383001092BD00CA
:1015400080918300843010F0109283008AE08093B1
:10155000C00080937A0010927B00909183009F5F7F
:1015600090937C0080937D0080937E0080937F0029
:101570008FE996E8A1E081509040A040E1F700C0DB
:1015800000001092C0006091830081E090E042D2A0
:101590001092BE000895AF92BF92CF92DF92EF9269
:1015A000FF920F931F93CF93DF9384B38F6384BB1A
:1015B00087B38C6387BB81B3886181BB85B583604A
:1015C00085BD89B7806C89BF82D880E061E041E049
:1015D000A8D580E390E062E370E041E350E025E0CD
:1015E00009D1E1D88093CC00882321F081E060E02C
:1015F00070E02AD787EA91E60197F1F700C0000072
:1016000082E090E0FFD1813061F080E090E061E025
:1016100001D281E090E063E0FDD182E090E061E002
:10162000F9D180E090E0EED18093840081E090E0F9
:10163000E9D18093830078948AE08093C0008093FE
:101640007A0010927B00909183009F5F90937C00C2
:1016500080937D0080937E0080937F008FE79AE1E6
:10166000A6E081509040A040E1F700C00000109239
:10167000C00087ED90E069EE70E040ED50E0A3D54A
:10168000C5E8D0E0CC24C3948E010F5F1F4F0F2E0E
:10169000FAE0DF2EF02D0F2EF9E7EF2EF0E0FF2E0F
:1016A000F02D0F2EF9E6BF2EF02D0F2EF8ECAF2EF9
:1016B000F02D8091C0008111E4DC68DEB09B23C076
:1016C0008091C0008823F9F48091BC00882389F7B9
:1016D0008091BC008F5F8093BC008091BD008F5FC4
:1016E0008093BD008091CF00873030F41882D801FC
:1016F000BC92F701A08205C0C882D801DC92F70134
:10170000D08209DCD6CF1092BC00D3CFE091ED009F
:10171000F091EE0090818091EC0089230895E09192
:10172000EA00F091EB0090818091EC00892B80839E
:10173000E091EF00F091F00090818091EC00892B16
:1017400080830895E091EA00F091EB009081809110
:10175000EC00809589238083E091EF00F091F00008
:1017600090818091EC008095892380830895E09199
:10177000EA00F091EB0090818091EC008095892344
:101780008083E091EF00F091F00090818091EC0077
:10179000892B808385EA95E08115910511F00197E9
:1017A000F1F72FB7F894E091EF00F091F0009081FD
:1017B0008091EC0080958923808386EC90E08115F0
:1017C000910511F00197F1F7E091ED00F091EE0035
:1017D00030818091EC002FBFAEEDB4E0A115B105D2
:1017E00011F01197F1F79081982311F08323089558
:1017F00081E008955093F0004093EF007093EB0068
:101800006093EA009093EE008093ED0081E090E019
:10181000AC0102C0440F551F2A95E2F74093EC003B
:10182000A6DF08952FB7F894E091EF00F091F00053
:1018300030819091EC00932B9083E2E0F0E0E11591
:10184000F10511F03197F1F7882351F0E091EF00A5
:10185000F091F00030819091EC009095932390836B
:10186000E6E2F0E0E115F10511F03197F1F7E091D2
:10187000ED00F091EE0030819091EC00392309F4F5
:1018800080E0E7E8F0E0E115F10511F03197F1F7BC
:10189000E091EF00F091F0003081909593239083D8
:1018A0002FBF08950F931F93182F08E0812F817089
:1018B000B9DF1695811110680150C1F7812F1F9172
:1018C0000F9108958FEFEEDF0895DF92EF92FF9270
:1018D0000F931F93CF93DF93D82EEB0148DF88231C
:1018E00041F580EFDFDFEE2410E40F2EF8EFFF2E3E
:1018F000F02DF10E81E096DF082F81E093DF882341
:1019000019F0002351F018C0002341F51D1508F10E
:10191000888180FF02C0D116F9F4802F83DF88818F
:101920008695888311501F1529F7112349F02196B8
:10193000DCCFEE24EA9404C00F2EFEEFEF2EF02D44
:101940008E2DDF91CF911F910F91FF90EF90DF903F
:101950000895E12E01E002C0E12E01E0802F62DF58
:101960008881869580688883DDCF0F931F93CF93FE
:10197000DF93082FEB01FBDE209741F085E592DF36
:1019800018E089918FDF1150E1F702C08CEC8ADFFB
:10199000802F88DFDF91CF911F910F910895991BC0
:1019A00079E004C0991F961708F0961B881F7A9556
:1019B000C9F780950895AA1BBB1B51E107C0AA1F58
:1019C000BB1FA617B70710F0A61BB70B881F991FE0
:1019D0005A95A9F780959095BC01CD01089597FB84
:1019E000092E07260AD077FD04D0E5DF06D00020B7
:1019F0001AF4709561957F4F0895F6F7909581954B
:101A00009F4F0895E199FECF9FBB8EBBE09A992727
:101A10008DB30895262FE199FECF9FBB8EBB2DBBC2
:101A20000FB6F894E29AE19A0FBE01960895F894E1
:021A3000FFCFE6
:101A320001030406090B0C0E002010300828183888
:101A420004243CFF0101FFFFFFFF0A0A0A0A0A0AF7
:101A5200000000020101FA01152A3F54697E93A891
:101A6200BDD2E7F5E7D2BDA8937E69543F2A15019E
:101A720069747F8A95A2AFBAC6D2DEEAF5EADED2EF
:0C1A8200C6BAAFA2958A7F7469FF01000C
:00000001FF
